:0C0000000C9454000C9400000C940000C0
:10000C000C9400000C9400000C9400000C94000064
:10001C000C9400000C9400000C9400000C94000054
:10002C000C9400000C9400000C9400000C94000044
:10003C000C9400000C9400000C9400000C94000034
:10004C000C9400000C94000080C00000003FCDCC4C
:10005C004C3D0AD7A33B6F12033A17B75138ACC5C6
:10006C00A736BD37063553696E2000436F732000E9
:10007C0054616E2000436F7420006153696E0061FF
:10008C00436F73004C6F67200053717274200065CE
:10009C007870200002008D0154000000F894EE27C7
:1000AC00ECBBF1E0FBBFEBBFE5BFF8E1F1BDE1BD9F
:1000BC008DE0A2E0BB27ED938A95E9F780E094E010
:1000CC00A0E6ED930197E9F7E0EAF0E085919591D0
:1000DC00009761F0A591B59105901590BF01F001C5
:1000EC0005900D920197E1F7FB01F0CFEFE5EDBF25
:1000FC00E4E0EEBFC0E6D1E00C948400EFE0E7BB97
:10010C00E7E0E4BBEFE0E1BBE0E1EA930E94CA0365
:10011C0002D0FECFFFCF1A930A9301E010E00E94A9
:10012C008A0639F40E9490060E9495060E949E064B
:10013C0085C0EAE07E1610F40E94B306E9E0E715EC
:10014C0018F4E0E17E1608F042C0EFE0E71519F470
:10015C000E94E20673C0672C0E94E506E1E0F0E025
:10016C00FA93EA933CD1002E012A89F10E948A0667
:10017C0019F40E94E20662C0EAE07E16E0F40E94E6
:10018C00EA060E94F306DF01CB01E72D0E94FA0676
:10019C000E9487090E9400070E94E5060E94090739
:1001AC000E9401040E9409070E949803E2E3F0E018
:1001BC000E940E070BC0EEE0E71541F4EDE3EA9365
:1001CC000E947E033ED0772400E010E0CCCFEFE01D
:1001DC00E71590F50E9468030E9490060E94950610
:1001EC000E9490060E9400070E9490060E9412072F
:1001FC000E94E506E2E0F0E0FA93EA93F0D0672C77
:10020C0001E010E0002E012AB9F00E948A0619F4D0
:10021C000E94E20613C0EAE07E1618F40E94B306B0
:10022C0008C0EEE0E71529F4EDE3EA930E947E03A3
:10023C0060D001E010E0E6CF0E9490060991199180
:10024C000895EAE0E61531F40E941B070E94230A88
:10025C000E941207EBE0E61531F40E941B070E9486
:10026C00D5090E941207ECE0E61541F40E94EA065B
:10027C000E942C070E9480090E941207EDE0E615EF
:10028C0031F40E941B070E9487090E9412070E94EA
:10029C0035070E942D040E9409070E944207089509
:1002AC000E9447070E944C0744245524E881F98199
:1002BC004E165F06A4F4A0916C01B0916D01809173
:1002CC006E0190916F01EAEEF7EE6DE270E40E9420
:1002DC00D5090E944C07F20131962F01E7CFE0912E
:1002EC006C01F0916D0160916E0170916F0122961D
:1002FC0008950E942C07A5E3BAEF8EE89CE30E94B8
:10030C00D509E0937001F0937101609372017093C1
:10031C007301E0E1E61531F40E9455070E944A058D
:10032C000E941207E1E1E61531F40E9455070E9484
:10033C00AE050E941207E2E1E61531F40E94550762
:10034C000E94B9050E941207E3E1E61551F40E94E0
:10035C0055070E94B9050E9460070E94230A0E945B
:10036C001207E4E1E61531F40E9455070E943506A8
:10037C000E941207E5E1E61531F40E9455070E9430
:10038C0075060E941207E6E1E61541F40E942C075F
:10039C000E94BC080E94D2040E941207E7E1E615F5
:1003AC0041F40E942C070E94BC080E9430080E9455
:1003BC001207E8E1E61551F40E942C070E94160979
:1003CC00FA93EA930E9456010E9412070E94350785
:1003DC000E942D040E9409070E9442070895A881DB
:1003EC00B981119721F5AA81BB811A9721F4EFE20B
:1003FC00EA930E947E03AA81BB811B9721F4EAE257
:10040C00EA930E947E03AA81BB811C9721F4EDE242
:10041C00EA930E947E03AA81BB811D9721F4EBE233
:10042C00EA930E947E03E4E6F0E00E940E07A881A6
:10043C00B981129711F00C946F02AA81BB8150976D
:10044C0021F4E2E7F0E00E946507AA81BB81519795
:10045C0021F4E7E7F0E00E946507AA81BB8152977F
:10046C0021F4ECE7F0E00E946507AA81BB81539769
:10047C0021F4E1E8F0E00E946507AA81BB81549762
:10048C0021F4E6E8F0E00E946507AA81BB8155974C
:10049C0021F4EBE8F0E00E946507AA81BB81569736
:1004AC0021F4E0E9F0E00E946507AA81BB8157972F
:1004BC0021F4E5E9F0E00E946507AA81BB81589719
:1004CC0021F4EBE9F0E00E946507E4E6F0E00E941D
:1004DC000E07249608951A9311E0103011F40C9421
:1004EC000F03909A919892989398849B03C0E7E09D
:1004FC00F0E08FC0859B03C0E8E0F0E08AC0869BEB
:10050C0003C0E9E0F0E085C0879B03C0EAE0F0E0BF
:10051C0080C09098919A92989398849B03C0E4E041
:10052C00F0E077C0859B03C0E5E0F0E072C0869BED
:10053C0003C0E6E0F0E06DC0879B03C0EBE0F0E0A9
:10054C0068C090989198929A9398849B03C0E1E02C
:10055C00F0E05FC0859B03C0E2E0F0E05AC0869BF0
:10056C0003C0E3E0F0E055C0879B03C0ECE0F0E093
:10057C0050C0909891989298939A849B03C0EFE006
:10058C00F0E047C0859B03C0E0E0F0E042C0869BF2
:10059C0003C0EEE0F0E03DC0879B03C0EDE0F0E06F
:1005AC0038C0A89AA998AA989D9B03C0E0E1F0E0F6
:1005BC0030C09E9B03C0E1E1F0E02BC09F9B03C0C9
:1005CC00E2E1F0E026C0A898A99AAA989D9B03C0E6
:1005DC00E3E1F0E01EC09E9B03C0E4E1F0E019C033
:1005EC009F9B03C0E5E1F0E014C0A898A998AA9AD3
:1005FC009D9B03C0E6E1F0E00CC09E9B03C0E7E1CD
:10060C00F0E007C09F9B03C0E8E1F0E002C011E0FE
:10061C0064CF19910895FFE0FA95F1F70895A7B307
:10062C00AF70A7BBC19AC0980E941103C29A0E94D6
:10063C001103A6B3C2980E941103C29A0E9411031F
:10064C00C298A7FDF1CF0895A07FAB2BA8BBC29A8F
:10065C000E941103C2980E9411030895C198A7B378
:10066C00A76FA7BBB8B3BF70A8810E942A03A8814B
:10067C00A2950E942A03C19A21960895C29A0E94BB
:10068C001103E6B3C2980E941103E07F08950E9403
:10069C0011030E944403AE2F0E944403C198E295BB
:1006AC00EA2B08950E941503E881F0E0E357FE4F12
:1006BC00E081A981EA0FEA930E9434039980888033
:1006CC00229608950E941503E2E0EA930E943403F7
:1006DC000E941503ECE0EA930E9434030E94150378
:1006EC00E1E0EA930E943403E0E08E2E9E2E089502
:1006FC00EF93FF93A8816894AA3021F0E894939427
:10070C00B91438F48394E0E0EA938A920E94580377
:10071C002EF085DFC09AA881AA93A0DFFF91EF91FC
:10072C00219608951A93A981BA81ED91A983BA8370
:10073C001E2FE03021F01A930E947E03F4CF188113
:10074C0010C01A93E981FA813196E983FA833197C3
:10075C00E4911E2FE03021F01A930E947E03F2CF19
:10076C00188123960895AA27BB271197F1F70895AE
:10077C00C198A7B3A76FA7BBB8B3BF70A8810E94DD
:10078C002A03C19A21960895C298C098B880E8812E
:10079C00E058E0938F01E881E054E09390010E94CF
:1007AC0069070E9469070E9469070E94B903E0E289
:1007BC00EA930E94BE030E94B903E8E20E946F070D
:1007CC00E4E00E946F07E5E80E946F07A7B3AF70E3
:1007DC00A7BBC19A0E944D03E53011F0E0E009C0BF
:1007EC000E941503E6E0EA930E9434030E9468031A
:1007FC00E1E021960895A991B991E991F99130968A
:10080C002AF4E095F09531966DE26D93E89480E1D1
:10081C0097E20DD088EE93E00AD084E6992707D0B2
:10082C008AE005D06E2F10D066276C93089566274A
:10083C00E817F90720F06395E81BF90BC9F7662355
:10084C0011F416F008956894605D6D9308952497E3
:10085C001A930A930E9474070E948C0A64F4E98527
:10086C00FA856B857C850E94E1080E9479070E94BD
:10087C007E07EDE2EC93A885A73010F0E6E0E88760
:10088C00E885A6E5B0E0F0E00E94A608EA0FFB1FA1
:10089C000E94B6080E9474070E9487090E9479077B
:1008AC0010E00E9447070E9485070E948A070E9459
:1008BC00680A40F00E948F070E94F3060E94850789
:1008CC001F5FF3CF103029F40E947E07E0E3EC9316
:1008DC0030C0E12F1150E03061F10E948F07E0E051
:1008EC00F0E060E271E40E94230AA0E0B0E080E056
:1008FC009FE30E9487090E94BC080E9495080E94F1
:10090C0085070E948A070E94230A0E9416090E2F4F
:10091C000E947E07E02FE05DEC93E02F0E948F0792
:10092C000E94FA060E94D5090E9474070E9494073F
:10093C00D0CFE885E03029F4AE81BF81E0E0EC93C4
:10094C0027C00E947E07EEE2EC93E885E150E88731
:10095C00EF5FD1F00E9474070E94F3060E947907A2
:10096C00E985FA856B857C850E9414090E2F0E94FF
:10097C007E07E02FE05DEC93E02F0E9474070E944D
:10098C00FA060E949407E1CFAE81BF81E0E0EC93C0
:10099C00198108812D96089524971A930A93C3D22E
:1009AC000E94900A2CF0EFEFFFEF6FE77FEF68C02B
:1009BC00BFD20E94BC08EDB7FEB73197FA93EA9309
:1009CC001F930F930E94CE080F911F91B6D2ABD2FA
:1009DC00B9D238F4ADD2A7D20E948709AED2015059
:1009EC001040A1D2B6D27F936F93FF93EF93A0D216
:1009FC0061D20E948709AF91BF918F919F910E9404
:100A0C00230A9BD295D28FD20E94D50978D2EA8143
:100A1C00FB816C817D81A6E2B2E485E69FE30E94B6
:100A2C00D509DF01CB01EEE4F1E164E570E497D286
:100A3C007AD20E94D5097F936F93FF93EF9369D27B
:100A4C00EDE4F1E164ED7FE38AD2AF91BF918F9138
:100A5C009F910E94230A7F936F93FF93EF93F8016A
:100A6C000E94B1080E944D09A8E1B2E781E39FE31F
:100A7C000E94D509AF91BF918F919F910E948709D8
:100A8C00198108812A9608956FD2E3E8F9EF62E2A2
:100A9C007EE30E94D50970D274D20E94BC080E94D9
:100AAC00950874D25CD268D276D20E94680A09F09A
:100ABC0010F40C9465056FD252D25ED211E066D25E
:100ACC00E0E0F0E060E87EE30E94680A09F010F4D0
:100ADC000C94740560D20E9480094ED2103009F03B
:100AEC0060D263D2E983FA836B837C8363D2A1EBFC
:100AFC00B4EC86E292E40E94D509DF01CB01EDE172
:100B0C00F5EE6DE272E42BD25AD2ACE4B3E584E09C
:100B1C0091E40E9487093AD20E94D5097F936F9382
:100B2C00FF93EF9347D2A1E1BDEE8EED9FE30E94C0
:100B3C00870945D2AEE5BBE788EA9FE30E948709A7
:100B4C00AF91BF918F919F910E94230A1881C5C0CC
:100B5C003DD2EBEDFFE069EC7FE30E9480090E943F
:100B6C00BC0892DFCFC0249736D2F2DFE883F9833A
:100B7C006A837B830E94880A59F434D20E94900ABB
:100B8C0014F435D235C0EFEFFFEF6FE77FEF30C0D5
:100B9C0022D27ADFDF01CB012FD20E94230A28C098
:100BAC002497EC81FD816E817F811CD20E94D50936
:100BBC00E883F9836A837B831FD2A5E6B0ED8BECC7
:100BCC0090E41FD20FD20E94D5097F936F93FF93AD
:100BDC00EF9312D2A0E0BDE689E291E40E9487096E
:100BEC00F5D10FD2AF91BF918F919F910E94230AA3
:100BFC0028960895EBD1EDECF3E164ED7EE30E94D1
:100C0C00680A18F4F9D106D27DC0E0D1EAE7F2E81F
:100C1C006AE170E40E94680A09F010F40C941D0655
:100C2C00EBD148D10E94230AF5D1F7D16BC0CED1BC
:100C3C0090D17F936F93FF93EF93DED13BD10E94C2
:100C4C008709AF91BF918F919F910E94230AE2D1A6
:100C5C00ABEDBFE089E49FE30E94870953C084D1C8
:100C6C00E1D148F093D10DD10E94680A19F010F02F
:100C7C000C94410603C0BBD118812FC087D10E94B0
:100C8C008C0A14F48ED111E090D114D168D10E9449
:100C9C00BC080E943008E983FA836B837C8376D18D
:100CAC0051D109F010F40C9463066BD1A981BA816F
:100CBC008B819C81BED1B1D103C07CD167D1B9D11C
:100CCC00E983FA836B837C83103029F073D10E9403
:100CDC00E108188102C06ED118812996089576D149
:100CEC00A1D148F073D1CDD00E94680A19F010F050
:100CFC000C94810602C07BD105C07ED10E94BC0839
:100D0C00AEDF8BD1249608950E9471027E2EEFE007
:100D1C00E7150895E0E0F0E060E070E00895E093FE
:100D2C006001F09361016093620170936301089517
:100D3C00F1DFE0936401F0936501609366017093B9
:100D4C006701E8DFE0936801F093690160936A0141
:100D5C0070936B010E946803DDCFA0916001B0918C
:100D6C0061018091620190916301E0E0F0E060E24A
:100D7C0071E40E94D509DF01CB01E72DFF2766271F
:100D8C0077270E944D090E948709C9DFE72DF0E003
:100D9C00FA93EA93E4E7F1E0FA93EA930E940104F0
:100DAC00E4E7F1E0FA93EA930E949803E2E3F0E0BF
:100DBC00FA93EA930C942408ADDFB1DFB9CFE72D99
:100DCC00F0E0FA93EA930895A0916401B091650163
:100DDC0080916601909167010895E0E0F0E060E297
:100DEC0071E40E94D5090895FF27662777270E9492
:100DFC004D090895E0936401F093650160936601D9
:100E0C00709367010895E4E7F1E0FA93EA9308958B
:100E1C00FA93EA930C942408E0936801F093690127
:100E2C0060936A0170936B010895E0916401F091F5
:100E3C0065016091660170916701A0916001B091AC
:100E4C00610180916201909163010895E0916001CC
:100E5C00F091610160916201709163010895E091DC
:100E6C006801F091690160916A0170916B010E94B7
:100E7C00BC08E3E0EA93C7CF0E949803E4E6F0E0F5
:100E8C00C7CFE0E0F0E060E87FE30895E0936C0109
:100E9C00F0936D0160936E0170936F010895E09172
:100EAC007001F091710160917201709173010E9457
:100EBC00BC080895A0E0B0E080E89FE30895FA93A1
:100ECC00EA930C94A7030E94B903E0E3EA930C9411
:100EDC00BE03EA930E9434030C94B903A985BA8526
:100EEC008B859C850895E987FA876B877C870895A5
:100EFC00AE81BF811196AE83BF8311970895EA83AB
:100F0C00FB836C837D830895EA81FB816C817D81F9
:100F1C00E5CFAA81BB818C819D8108950E94C10877
:100F2C000E948009E0CFAE81BF81888599850895A4
:100F3C00EE81FF81688579850895EE83FF8368874C
:100F4C0079870895E3EFF4E065E37FE30E94680A94
:100F5C00089597DF0E94C1080E94800908950E949D
:100F6C00C1080E948009089524971A9310E0AD815E
:100F7C00BE818F8198850895ED83FE836F8378877A
:100F8C000895ED81FE816F8178850895AD81BE81D4
:100F9C008F8198850895FADFE0E0F0E060E07FE370
:100FAC000895EFDF0E94E108E7CFEBDFEFDF0E944F
:100FBC00D5090895E981FA816B817C810895A98115
:100FCC00BA818B819C810E94D5090895A881B98131
:100FDC008A819B810895EC81FD816E817F810E94C5
:100FEC00BC080895AC81BD818E819F810895EFEF7F
:100FFC00FFEF6FE77FE70895E881F9816A817B81D4
:10100C0008950E94D509AEE4BFE88AE491E40E94F9
:10101C00870908950E94BC08C3CDABEDBFE089ECF5
:10102C009FE39DCFE0E0F0E060E87FEB0E94680A70
:10103C0008950E94230A0E94BC08DCCDE991F99125
:10104C00309639F088EE93E00197F1F7A895319737
:10105C00C9F7089524975F939F81992311F42896DB
:10106C008CC112F4289695C14F9342E48E81BD81B8
:10107C00AC8188839983AA83BB83FD01BC01AC81BD
:10108C00BD818E819F81D9D188819981AA81BB81B3
:10109C0038D1BBD07A959FD088819981AA81BB81A8
:1010AC00AE27A87F21F4BF178607970729F04A952A
:1010BC0019F0DF01CB01DDCF4F915F912896089598
:1010CC007B816A81F981E88177FB770F67FD71601D
:1010DC00972F9E5781F078F0983190F4AA27BB2770
:1010EC00882708948795B795A7959A95D1F7EA2301
:1010FC00FB23682305C0E8947727EE27FF27662794
:10110C006F77769508F4606877F9A991B991899110
:10111C009991EA17FB076807790797FB0895D0DFC9
:10112C0009F40895F6F79FEBAA27BB2780E8E9C0DE
:10113C00F09560957095E195FF4F6F4F7F4F089537
:10114C00EE0FFF1FEE0FFF1F0895FE2FFF0FFF0B7B
:10115C006F2F7F2F08956F2F660F660B762F0895D4
:10116C000590159065917491F00108957A936A93A6
:10117C00FA93EA930895182E862F612D192E972F26
:10118C00712D1B2EBF2FF12D1A2EAE2FE12D089590
:10119C00A991B991E991F9916991799177FB660FD0
:1011AC00771F88277E57880B7D938C937EE77695E7
:1011BC0067950EF0089530976040704009F07058B4
:1011CC000895552342F4503811F4E0FF04C03196D1
:1011DC00691F791F6BF050E8572711F45F93CDC04E
:1011EC005F3F31F0660F000C57956795752F08958A
:1011FC005F9300200AF0CDC0C6C050E8192E15220E
:10120C00880F991F9527550F879550E8072E0522B3
:10121C00660F771F7527550F67950895689401C061
:10122C00E8945F93F2DF703818F07F3F08F4A5C0A4
:10123C0056E1571BAAF4519558300EF4593030F042
:10124C00EFEFFFEF6FEF7FE777F91AC077275523A2
:10125C00B9F0EE0FFF1F661F771F5A95D1F710C01C
:10126C007727583028F0EF2FF62F672F5850F9CFEB
:10127C00552331F076956795F795E7955A95D1F703
:10128C0000200AF455DF5F910895689401C0E8943A
:10129C00309760407040B1F0002426F0772312F4B0
:1012AC00009446DF172E7EE1112032F07A95EE0F76
:1012BC00FF1F661F111CF9CFEF2FF62F612D5F93C7
:1012CC008ADF5F9108954F93AF01FD01DA01AB0105
:1012DC00BC01CA01402D012C142E4F910895EA0F28
:1012EC00FB1F681F0895E095F0956095EF5FFF4F29
:1012FC006F4F08955F9381DF903871F150E8152698
:10130C0004C05F937ADF903839F1703821F1572F90
:10131C00591B13F112F4D7DFFACF583118F0AA2762
:10132C00BB278827583028F0AB2FB82F8827585068
:10133C00F9CF552329F08695B795A7955A95D9F7E6
:10134C00502D512562F0CBDF38F46795F795E79572
:10135C00739513F41EC0B7DF3EDF5F910895EA1B4F
:10136C00FB0B680B51F010F40094BDDF6623A2F365
:10137C00EE0FFF1F661F7A95CBF7EE27FF27662728
:10138C0077275F910895EFEFFFEF6FE77FEF5F91A6
:10139C000895EFEFFFEF6FE77FE75F9108955F939D
:1013AC002CDF703851F3903841F301240894791FE5
:1013BC0023F41CF300203AF3ECCF0F921F932F93DE
:1013CC003F934F93112722279927689FA0018F9F46
:1013DC00302D410D591F6B9F300D411D591F8E9F94
:1013EC0027D0BF9F25D06A9F23D0BE9F1DD0AF9F13
:1013FC001BD0AE9F110D291F391F491F591FE32FF9
:10140C00F42F652F522F4F913F912F911F910F90D9
:10141C0066232AF0550FEE1FFF1F661F02C073953F
:10142C004BF2CFDE5F910895100D211D391F02C0C4
:10143C00200D311D491F591F08955F93DEDE703852
:10144C0021F411200AF49FCFA4CF903809F495CF42
:10145C0001240894970B1BF4D4F30020F3CF792FBD
:10146C001F932F933F934F93112411272227332738
:10147C004427552790E2AE17BF078607410730F087
:10148C00AE1BBF0B860B410B089401C08894551FF3
:10149C00221F331F111CAA1FBB1F881F441F9A95A4
:1014AC0051F7F901612D4F913F912F911F916623B7
:1014BC0032F0550FEE1FFF1F661F7A9543F281DE47
:1014CC005F91089599239AF0772342F0971748F08B
:1014DC0029F4AE17BF07860720F031F09894889452
:1014EC0008959894089408951894889408957723EF
:1014FC00C2F7971798F3A9F7EA17FB07680788F361
:10150C0099F3ECCF3097604070400895109780406D
:10151C009040089500240A160B0608060906089543
:00000001FF
